:020000020000FC
:1000000069CDA4C1000000001FC000008DC0000029
:10001000000097C00000000000000000020304067A
:10002000080C10182030406080000406080C1018DE
:100030002030406080A0C0000003070F1F000505AE
:100040000D050305030302004FB662FD0CC05520E9
:1000500041F00994C52DC095089483FDC795C4BD92
:1000600064604FBE1895C0916400089483FDC795E5
:10007000C4BD6B7FC0916400CF3F09F41EC070FF08
:100080001AC082FD05C04FBE91989098939818951C
:1000900076FD0EC064FD0CC0C091B100C0FD949807
:1000A000C1FD9798C2FD9598CAEFC095CA95F1F722
:1000B0009198909893984FBE189524BCCC27C06413
:1000C000C8BF6460F8CFC6CF70FFC4CF64FDC2CF95
:1000D000919AC0CF70FFBECF64FDBCCF909ABACFCB
:1000E00070FFB8CF64FDB6CF939AB4CF949A70FFE7
:1000F000B1CF64FDAFCFC7E0CA95F1F7919AAACF0F
:10010000979A70FFA7CF64FDA5CFC7E0CA95F1F716
:10011000909AA0CF959A70FF9DCF64FD9BCFC7E0CA
:10012000CA95F1F7939A96CF4FB6C9B7CF7EC9BF9C
:100130006E7FCCB5CE0DDDB5DF1DDBBDCABD4FBEBC
:1001400018953FB68F7EABB7A074A2118061A0E076
:10015000ABBFA9B7AE7FA9BF7894A0916800AA23CE
:1001600041F085FD2EC0A0916800AA95A09368007B
:1001700028C040E050E085FD14C0A0B396FDA095D6
:10018000A2FD4FEFA3E096FDA2E0A5BFAA27A064C1
:10019000AABF8D7FA0B396FDA095A2FD5FEF451786
:1001A00041F7A8E161FDA093680085FD03C0A8E1C7
:1001B000A0936800409396008160442311F0209240
:1001C000990085FD0EC0A0916900AA2331F0A0918D
:1001D0006900AA95A093690004C08061AA27A06461
:1001E000AABF80FF3DC0A09196004A2F61FF8E7F7D
:1001F00085FD18C0403F08F040EFA42FA295AF70D6
:100200004A0F5091B600533069F0A695A69550FD5F
:1002100001C0A69552FD03C0A41B4A2F03C04A0F7C
:1002200008F44FEFA0919F004A1708F44A2F40931B
:100230006100A72FA670A1F073FD12C0A0917000FD
:10024000AA0FAA0F50919E0056955695541708F084
:10025000452F4A0F4093610018F4AFEFA09361005F
:10026000A0916100A093630040916300A0919B0066
:100270004A1708F04A2F542EA091A000AA2309F48F
:1002800022C0542F5A1B10F4A42F50E0BA2E889489
:10029000AA1FAA2EA091A200A095AA22A50E58F0EE
:1002A000A091A100A21509F0AA95AA0EA093A10001
:1002B00048F04A2D08C0A091A100BA1608F0A395F5
:1002C000A093A1004FEF409364007F7B485F08F04C
:1002D0007064A0916000A395A093600051F0F89421
:1002E000A9B7A160A9BF84FF02C0A0E4ABBF3FBE15
:1002F0001895A0917400A395A093740041E05091CB
:100300006800552329F085FF03C05A955093680073
:10031000A0919600A13018F0209299000DC0209273
:100320009A002092A300A0919900AF5FA09399003A
:1003300018F0AFEFA0939900F894A9B7A160A9BFF6
:1003400084FF02C0A0E4ABBF3FBE18953FB64CB5DA
:100350005DB58F7EABB7A074A2118061A0E0ABBF8A
:10036000A9B7AE7FA9BF789481FD23C0A2E096FD16
:10037000A3E0A5BF8260A0B396FDA095A2FF05C033
:1003800040936500509366003EC1A3E096FDA2E055
:10039000A5BFAA27A064AABF8D7F85FF01C026C183
:1003A00040E0A0B396FDA095A2FD20C14093960029
:1003B0000FC1A3E096FDA2E0A5BF8D7F61FF71C0D4
:1003C000A2E096FDA3E0A5BFAA27A064AABF826011
:1003D0004093910050939200A0908F004A19B090E2
:1003E00090005B09BB24A22C4C38520518F42092D3
:1003F000950049C0A091D400AA2359F1483C520568
:1004000028F4A0E1BA2EAAE0AA2E23C04836A1E023
:100410005A0728F4A8E0BA2EAFE0AA2E1AC0403D31
:10042000A2E05A0728F4A4E0BA2EAEE1AA2E11C029
:10043000403AA5E05A0728F4A2E0BA2EACE3AA2E6F
:1004400008C04839A8E05A0720F4A1E0BA2EA8E76E
:10045000AA2EC42EA0919300CA1AD52EA091940062
:10046000DA0ADD202AF4AFEFC094D094CA1ADA0A6F
:1004700020929500A8E0A210A0E0CA14DA0618F4B1
:10048000A1E0A09395004093930050939400409175
:1004900091005091920040938F005093900042E061
:1004A00097C0A09165004A1BA09166005A0B94FD6D
:1004B00082C093FD80C092FD7CC086FF03C0D52E14
:1004C000C42E0CC05695479591FD73C0569547951F
:1004D00090FD6FC0D52EC42ED694C79461FD19C06F
:1004E000AC2DAC51AD2DA24008F005C0DD2089F443
:1004F000AC2DA85C70F4A0916700A395AA2311F01D
:10050000A0936700AA3008F471C020929600816021
:100510006DC0A0916700AA2319F0AA95A093670067
:10052000A22C5091BA0097FD06C0A090C80053308D
:1005300011F4A090D000AAEFAA0EA22DA21DCA18F5
:10054000DA0A4FB74170533049F4442321F087FD54
:1005500005C0806803C087FF01C08F77442359F02E
:10056000533031F4AFEFC094D094CA1ADA0A03C002
:1005700040E050E020C0533049F4CC0CDD1CAAE030
:10058000CA1AD20818F4A0E0CA2ED22CAFEFCA16AD
:10059000D20418F04FEF50E00EC0A091AC00CA9EFC
:1005A000412D000C441F50E008F012C04FEF50E006
:1005B0000FC05695479594FF07C0552309F04FEF9C
:1005C000A42FA6954A0F521D4F3F520508F04FEF3A
:1005D00040939600816061FF09C0AFE1A095A92317
:1005E000AB299A2F8F7DBB2009F48062A8E1A093EC
:1005F000680085FF03C0AAE0A093680061FD03C006
:1006000085FD01C08F7E85FD03C0A6E0A093690033
:10061000F894A9B7A160A9BF84FF02C0A0E4ABBF52
:100620003FBE189511E00AC013E008C01AE006C0EA
:100630001EE104C014E602C018EC00C005E1BB27AF
:10064000BA95F1F70A95D9F71A95C1F708952AE3F3
:1006500038E709C020E33CE806C02AE234EB03C0D7
:1006600025E238EC00C0B091AD00BA9509F40895C8
:1006700012E0BB27979ABA95F1F7909ABA95F1F7DD
:100680009098BA95F1F79798BA95F1F7123009F06A
:10069000919A123009F4939AB091AD00BA95F1F79E
:1006A000123009F09198123009F49398B7E8BA958E
:1006B000F1F71A95F1F6022FB22FBA95F1F70A95D4
:1006C000D9F73A9581F6979A0895221B39E0001FD1
:1006D0003A9509F40895221F211B18F4210F8894DC
:1006E000F6CF0894F4CF622C722CB0E08894B395C6
:1006F000221F331FE0F7379527958894912E802E7F
:10070000020B130B10F4192D082D10F4889401C05E
:100710000894661C771CBA9571F7172D062D08955D
:10072000322D11232AF43A9500951095031B130BD3
:10073000F894029F712C002D129F912C802C78949C
:10074000780C172D921C292DB4E06B2E2695179549
:1007500007956A94D9F7332321F000951095031B70
:10076000130B0895089510917B00169500917A005F
:100770000795B0917E00B01B0B2FB0917F00B10B9D
:100780001B2F28F40038BFEF1B0740F009C00F37BC
:10079000120508F405C00FE710E002C000E81FEFE3
:1007A0000093830010938400089500918300B0911A
:1007B00080000B0F10918400B09181001B1F20E07E
:1007C0003091840033230AF42A95B09182002B1FC4
:1007D0001AF4203F40F00AC02F3008F407C00FEF92
:1007E0001FEF2FE003C000E010E020EF3091630026
:1007F000B0919B003B1718F4323030F009C0B09133
:100800008400BB235AF004C0B0918400BB2332F4AF
:10081000009380001093810020938200089520911E
:10082000D70000918300000F10918400111F78DF22
:1008300011232AF40038BFEF1B0740F009C00F371F
:10084000120508F405C00FE710E002C000E81FEF32
:10085000002352F0B0916200B01B0B2F18F0013052
:1008600008F00AC001E008C000950F5FB091620077
:100870000B0F08F001C00FEF009385000895209141
:10088000D80000918100109182004ADF11232AF4E0
:100890000130BFEF1B0740F009C00F3F120508F4FD
:1008A00005C00FEF10E002C001E01FEF112352F06E
:1008B000B0918500B01B0B2F18F0013008F00AC072
:1008C00001E008C000950F5FB09185000B0F08F0A4
:1008D00001C00FEF0093630008950FEF71FD1EC07C
:1008E000B091D300BB23D1F0B0917B00BB23B1F01A
:1008F0000FEF10917B00E9DEF894B091730072FD68
:10090000B5E00B9F112D002D7894112309F00FEF06
:10091000B0919E000B1710F400919E0000939D0073
:10092000089500917A0010917B0000541140B0911D
:100930009D0010F4BA9501C0B39511F0B0939D00DD
:10094000089500C008952091B500B6B1B6FDFBCF63
:1009500004B115B1B6B1BF77B6B9B091AA00B395DD
:10096000B093AA00B83060F12092AA00B091D200F2
:10097000BB2321F1112329F0B091AB00BF3F61F0FF
:1009800009C0B091AB000B1739F020F4BB2321F064
:10099000BA9502C0B395E1F300919B00B093AB0010
:1009A000B03050F400ECB03038F400E8B03020F44F
:1009B00000E4B03008F400E000939B007F7E0895CF
:1009C000B0919B00B39511F0B0939B00B091AA0039
:1009D000B73009F47061089502E3F894B091D9003A
:1009E0000B9F012D000C001F7894B0919B000B17FA
:1009F00010F000919B000093610000936300502E63
:100A00000093640000939E00089520927A00B0EF56
:100A1000B0937B000895F8940CB51DB52091740037
:100A20007894309175006090760000937500109373
:100A30007600031B160971FD03C077FD80C028C036
:100A400070907700209377002709222319F00FEF89
:100A50001FEF0EC08090780090907900309378005E
:100A600060927900009175001091760008191909BB
:100A700020917A0030917B0036952795020F131F45
:100A800010F40FEF1FEF00937A0010937B002BC040
:100A900020917A0030917B003901B4E08B2EB2E0D6
:100AA0009B2E343040F08A949A94383020F072FDB6
:100AB00002C08A949A94769467948A94E1F72619EE
:100AC0003709992021F0169507959A94E1F7200FA0
:100AD000311F20937A0030937B0028F43FEF30934E
:100AE0007A0030937B00323008F4706871FF02C0E6
:100AF000B3E00DC0B091C40000917100023838F02D
:100B0000B395003A08F0B395B63008F0B5E09B2EE7
:100B1000B4E08B2E10917B0000917A0024E01695B2
:100B200007952A95E1F70819120928F0B02FB2505D
:100B3000B12FB20910F402E010E0980126C0209114
:100B40007A0030917B0039017694679466946694BC
:100B500066942619320906950695200F321D2093BA
:100B60007A0030937B00323008F07F7704E03695CE
:100B700027953695279526952695201B10F022302F
:100B800008F422E089019090C40060FDFECFE0905F
:100B90008B00F0908C006160B9B7B061B9BF3801CB
:100BA00077FD41C07694679400938B0010938C007E
:100BB000B92DB330E1F0B0FD04C0060D171D93014F
:100BC00006C0000F111F0250120922E030E0B92DBB
:100BD000B33068F020938D0030938E00009387002F
:100BE000109388006092890070928A003AC0009346
:100BF0008D0010938E0020938700309388006092C0
:100C0000890070928A0071FF0DC0BFE0B0938D0023
:100C100020928E00B093890020928A00B0938B00BE
:100C200020928C001EC0669400938B00B92DB330C7
:100C300091F0B0FD03C0060D262D03C0000F025039
:100C400022E0B92DB33038F020938D000093870057
:100C50006092890006C000938D0020938700609207
:100C6000890000917C0002FD0350013031F495FDB4
:100C70000CC0B2E0B06CB7B90BC0023021F4B3E0E5
:100C8000B06CB7B905C095FDF4CFB4E0B06CB7B99E
:100C90000091A200000F10F4BBE60B270093A20006
:100CA00060FDFECFB2E0B0936E006160B9B7B06195
:100CB000B9BFB72FB670D1F020917A0030917B0088
:100CC000369527953695279571FF02C0B0E43B0F06
:100CD000F8940CB51DB5020F131F1BBD0ABD616052
:100CE000B0E1B8BFB9B7B061B9BF78940895686092
:100CF00020927D0020E066FD20E206C06860209220
:100D00007D0020E266FD20E001E011E077FD11C0EA
:100D1000B72FB67009F0677F14E100917B0006954C
:100D200009F403950F3008F00FE071FF02C004E1F1
:100D300014E160FD0FC0B0917D00BB2359F071FF3D
:100D400006C0B0916E00BA95B0936E0011F4706257
:100D50004FC0ABDFB0B7B77FB0BFB8B1B0B7B86006
:100D6000B0BFB0917D00B395B0937D00B8B177FD71
:100D700006C0B1E071FDB3E0BA95F1F7B8B1B07259
:100D8000B21709F02AC071FF05C00395011708F0DA
:100D90000A95CFCF63FD05C00395011708F0B4CFC6
:100DA000C8CF677FF8943CB56DB470907A00B0916D
:100DB0007B00770CBB1F08F4BFEF770CBB1F08F458
:100DC000BFEF370D6B1E6BBC3ABD6160B0E1B8BFC1
:100DD000B9B7B061B9BF789497CFB0916D00B13019
:100DE00008F492CF63FD90CF0A9509F0A2CF7F7DE2
:100DF00020918D0030918E00F894B0E1B8BF0CB511
:100E00001DB5020F131F1BBD0ABDE0908700F090B7
:100E100088006160B9B7B061B9BF7894B72FB67078
:100E200039F0B0916D0072FFB395B0936D0009C0B9
:100E300075FF07C066FD05C063FD03C0BF91BF918C
:100E4000FDC4089500E063FF01C001E0F894109133
:100E50007100B7E01B9F212D102D7894200F26954F
:100E600017952695179526951795109371001837A5
:100E700018F4B8E7B093710000917100B09172005E
:100E80000B1720F0606191989098939860FDFECFC9
:100E9000E0908900F0908A006160B9B7B061B9BF95
:100EA0000895B2E095FD0AC0F894B0937C00979A3B
:100EB000949862FF01C0939A7894F4C0F894B09328
:100EC0007C00979A959862FF01C0919A7894EAC045
:100ED000B3E082FF24C095FD11C002E0F894B09306
:100EE0007C00E0E8F0E00093B1009398959A62FFEF
:100EF00002C0909A01C097987894D4C002E0F89408
:100F0000B0937C00E0E8F0E00093B1009198949AEF
:100F100062FF02C0909A01C097987894C3C095FD73
:100F20000BC0F894B0937C00EAE6F0E0939862FF7F
:100F300001C0909A7894B6C0F894B0937C00EAE629
:100F4000F0E0919862FF01C0909A7894ABC0B4E051
:100F500095FD0AC0F894B0937C00949A959862FF2E
:100F600001C0909A78949EC0F894B0937C00959AB2
:100F7000949862FF01C0909A789494C0B5E082FF83
:100F800024C095FD11C001E0F894B0937C00E6E721
:100F9000F0E00093B1009098979A62FF02C0919A96
:100FA00001C0949878947EC004E0F894B0937C00DB
:100FB000EAE8F0E00093B1009098979A62FF02C0CF
:100FC000939A01C0959878946DC095FD0BC0F894E4
:100FD000B0937C00E4E6F0E0909862FF01C0919A43
:100FE000789460C0F894B0937C00E0E7F0E09098CB
:100FF00062FF01C0939A789455C0B6E095FD0AC08F
:10100000F894B0937C00959A979862FF01C0919AEA
:10101000789448C0F894B0937C00949A979862FFB3
:1010200001C0939A78943EC0B1E082FF24C095FD40
:1010300011C004E0F894B0937C00EAE8F0E000937B
:10104000B1009198949A62FF02C0939A01C095985A
:10105000789428C001E0F894B0937C00E6E7F0E0D3
:101060000093B1009398959A62FF02C0919A01C0D3
:101070009498789417C095FD0BC0F894B0937C00B9
:10108000E0E7F0E0919862FF01C0939A78940AC07B
:10109000F894B0937C00E4E6F0E0939862FF01C01E
:1010A000919A78946F7E089523E630E0F9012092BA
:1010B000B100919890989398949A979A959A6B7F8B
:1010C0000895A2EBB0E00FEF0D930D930D930D93E8
:1010D00003E00D9304E00D9309E00D9303E00D93FD
:1010E00001E00D9301E00D93AEEBB0E001E00D9354
:1010F0000FEF0D930D930D930D930D9303E00D934F
:101100000FEF0D930FEF0D930D9305E20D9300ED8F
:101110000D930AEF0D930AEF0D9304E00D930FEF7B
:101120000D9301E00D9300E00D930AE70D930FEF8F
:101130000D9300E00D9301E00D9300E00D9303E0AB
:101140000D9300E00D9308952091B9008B7F23301B
:1011500009F48460B091BA00B33019F09F7DB1FDFD
:1011600090629F7BB091BB00B1FD9064223011F082
:10117000886001C0877F08950A95E00FF21DB49141
:101180000895ECE1F0E00091B200F6DFB093D700F3
:10119000ECE1F0E00091B300EFDFB093D800EAE2B9
:1011A000F0E00091B800E8DFB093D9000091B800FA
:1011B000023008F402E000937300B091CE000FEF0C
:1011C000B23009F400EAB33009F402E80093720087
:1011D000E8E3F0E00091D500CFDFB093A0000895E0
:1011E00008952091C8003091C900B091BA00B33081
:1011F00009F43E5097FF02C020E03FEFB32FB21B2F
:101200006B2EB25810F4B2E86B2E00E00395609E8E
:10121000B12DBD57D8F30093AC0008959068E1DF7D
:1012200007DA06DA20E030E0B0E16B2EFDD9B091AC
:1012300096002B0F321D6A94C9F7B4E036952795B6
:10124000BA95E1F7822E9F77CCDF0895F894E3E01A
:10125000F0E0B9E0B7BFB491B078C1F3F894A895C5
:10126000B1B5B861B1BDB0E0B1BDB4E0BEBFBFE5DE
:10127000BDBF1ADFB0E0B8BBB0E1B7BBB0E0B5BBF3
:10128000B0E0B4BBB0EBB2BBBBEBB1BB2224A0E07F
:10129000B0E02D92AA31E9F7A0E6B0E00FEF2D9271
:1012A0000A95E9F7B1E0B093A2000BDF03D3B7E0F2
:1012B000B06CB7B9B6B1B460B068B6B90091CA0045
:1012C0000093AD00B1E0B0936A00F894B5D9BFD9EE
:1012D000AFD9C0D9ADD9C1D9ABD973D3ADD9ACD9F8
:1012E000A9D9F8940AEF1AEFA0B396FDA095A2FF32
:1012F0001FC01A95C9F70A95B1F7E0E0FCE1B59176
:10130000B43E39F4B591B03E21F4B591BF3F09F434
:101310000CC0E0E0F395F395B591B83F49F4B59171
:10132000B43931F4B591BA3A19F4EE27F695099427
:101330000BDF27DF55DF55DF0091CA000093AD00BA
:10134000B3DEB2E0B3BFB2E0BEBDB2E0B5BDB1E561
:10135000B8BFB9BFB0B7B77FB0BFB8B1B0B7B860AA
:10136000B0BF60D97894EDDA20927000B3E096FDBA
:10137000B2E0B5BFB0E4BBBFBB27B064BABF8D7FDE
:101380005BD9626033E02CE0B0919500BB2321F47F
:101390002CE03A9509F4A5CF4BD980FFA2CF8E7FE0
:1013A000B0919600B23078F3B92FBF7100919800D8
:1013B00000939700B0939800B01729F72A9521F76A
:1013C0006D7FB3E096FDB2E0B5BFBB27B064BABF96
:1013D0008D7FB091D400BB2321F48062B92FB0700F
:1013E0009B2F8F7B2092670025D985FF05C0B09188
:1013F0006700BA3008F0806417D902E085FF01C0A9
:1014000000E0B0919600B017B8F3F89420D91FD936
:101410001ED9789411D920928600B091BA00B330C9
:1014200009F47EC001D9B091BE00B13008F478C093
:10143000B0916A00B13008F473C085FD18C0B09156
:101440009600BF3F08F46CC0F8940AD97894F2D89B
:10145000B0919600B130C0F7F894F9D8E7D8F7D832
:101460007894E8D8B0919600BF3FB0F3DCC2B8E002
:101470009B2E9068F894B5DE7894DCD8F8949F772A
:10148000B0DE80909600B0919600BF37789408F453
:101490004FC0C8D8F894E4D878949A9451F7BEDE37
:1014A000B82DB550B093C900C7D8F8948FD27894AE
:1014B000BAE09B2E9068F89494DE7894BBD8F894A8
:1014C0009F778FDE80909600B0919600BF3778941A
:1014D00078F7A8D8F894BBD8A9D8B9D878949A94B2
:1014E00049F79CDEB82DBB5FB093C8000B2F10915D
:1014F000C900125810F0100B20F4B2E80B0F009343
:10150000C9009AD8F89403D270D2789493D8F894FA
:1015100068DE7894B0919600BF3F08F48ECF83C206
:1015200000919600B09186000B1710F00093860092
:1015300081D801E0B091BA00B35009F405E0B09150
:101540009600B01708F069CFF8948AD889D888D85F
:10155000789472D820926A0020926B0020926C00DE
:10156000B0916B00B395B0936B00BF3F71F5B09134
:101570006C00B395B0936C00B091CC0009E1BA95C2
:1015800059F002E3BA9541F00DE7BA9529F00AEF58
:10159000BA9511F020926C00B0916C00B017A8F0D1
:1015A00083DD40D8B0916C00BA95B0936C00209266
:1015B0006B00B091CB00B093AD00F89451D8789403
:1015C000B091CA00B093AD0035D830D8B091680062
:1015D000BB2319F485FF01C084CE01E085FD01C065
:1015E00006E0B0919600B01708F4BACFB091BA00F7
:1015F000B35009F01FD8B0916800BB2309F471CE35
:10160000F89452DD209261002092620020926300E3
:10161000522C209264002092A1007894B091B700DF
:10162000BB0FB0939F0020927E0020927F002092FB
:10163000800020928100209282002092AA0060E027
:1016400070E020927100B8E0B093AA007061EAD710
:10165000B7E074FDB7E0B06CB7B9B6B1B068B064CC
:10166000B6B9B6B1B6FDFDCF04B115B1B6B1BF770D
:10167000B6B9112309F00FEF0093AB0064D9B8E0BD
:10168000B093AA00706160DDF894BFEFB0939B0047
:10169000A3D9B0916100B0939B00B0939C00B0932C
:1016A0009D007894B1E0B0936100B09363005B2E2D
:1016B000B0936400B093A400B0919A00B093A300DB
:1016C000B091BA00B33019F49F7D87FD90627160CC
:1016D000726020926D0091DCA7DC97D99CD995D9D6
:1016E0009AD993D90BDB3ED8ADDBDBDB94D9FFDA9B
:1016F00065FD39D877FFF1D877FD13D9A3DBE8DB97
:101700008AD9FCDA65FD51D89DDB21DC84D9EFDA7A
:1017100065FD85D897DB32DC7ED9F0DA65FDAFD880
:1017200091DB6BDC78D9E3DAB7E074FDB7E0B06C3D
:10173000B7B9B6B1B068B064B6B984DB75DC6BD943
:1017400002D971FF21C0B0919E00B0939B00B0936D
:101750009C00B0919A00B093A300B1E0B093A400B4
:1017600018E12CE0B0916D00B11740F07D7F7460FE
:1017700020936F00BFEFB0939B0006C0B09196001E
:10178000B13008F0AFCF64C072FF15C066FD13C062
:10179000B0916F00BA9519F47B7F7860A3CFB093B6
:1017A0006F00B0919600B13008F09CCFB091BA00B4
:1017B000B33009F04DC020927000B091990002E85A
:1017C0001091D600112309F003E0B01708F040C0D3
:1017D00085FF04C0B0916800BB23D1F1B091BA007D
:1017E000B33081F495FD03C087FD04C00BC087FFB3
:1017F00001C008C066FD06C06064B0919E00B09351
:101800009B0085CF00EF66FF05C0B0919E00B093AE
:101810009B0000E2B0917B00B01708F463CF66FF35
:1018200017C06F7B9F7D87FD90627460B2E1B093BB
:101830006F00B0919E00B0939B0054CFB0917000A8
:10184000B395B0937000B0919600BB2309F002C02D
:1018500020927000F89428DC8090B900B2E0B09338
:10186000B90072DC8092B90020926100209262007F
:1018700020926300522C2092640020929F0060E02E
:1018800070E07894D7D610DC0091D600002319F0D0
:10189000919A909A939AB7E0B06CB7B9B6B1B46028
:1018A000B068B6B985FF05C0B0917000B43008F0DB
:1018B00018CD52CEEDE0F0E023D00A3509F01BC080
:1018C000EEE0F0E01DD0053A09F015C03AE0A2EBD9
:1018D000B0E0E3E0F0E014D00D9331963A95D9F7FB
:1018E00039E1AEEBB0E0EFE0F0E00AD00D933196D5
:1018F0003A95D9F702C0E5DB0AD0E8E2F0E00895B6
:10190000E199FECFEEBBFFBBE09A0DB308951ED068
:101910003AE0A2EBB0E0E3E0F0E00D910FD03196B9
:101920003A95D9F739E1AEEBB0E0EFE0F0E00D9198
:1019300005D031963A95D9F712D00895E199FECFA6
:101940000DBBEEBBFFBBE29AE19A0895EDE0F0E03B
:101950000FEFF4DFEEE0F0E00FEFF0DF0895EDE0E1
:10196000F0E00AE5EBDFEEE0F0E005EAE7DF0895FE
:101970003091AE000091AF00313011F40093B60009
:10198000323011F40093B700333011F40093B800F3
:10199000343011F40093C400353011F40093B900D1
:1019A000363011F40093D500373011F40093CE0097
:1019B000383011F40093BA00393011F40093BB00B1
:1019C000089525E039D62A95E9F7089540D642D6FC
:1019D00044D646D62BD63BD63DD63FD641D626D684
:1019E00036D638D63AD63CD608953AD636D632D6FA
:1019F0002ED61CD635D631D62DD629D617D630D6EA
:101A00002CD628D624D608958090AE009090AF00B2
:101A10001ED61DD61CD60AD68A94D1F721D606D654
:101A20009A94E1F70895F894D1DF7894CADFC9DF7A
:101A3000B1E0B093AE00B1E0B093AF002092B0003F
:101A4000F894E2DF7894B5E06B2E70909600F4D5B0
:101A5000B09196007B16C9F7B13018F0BF3F40F146
:101A600007C086DFF89453DFB1DFB8E0B1BDA9DF6E
:101A70006A9459F7B091B000B395B093B000B33009
:101A800008F4DECF9EDFB091AF00B395B093AF0006
:101A9000F894B091AE00BA95EEE3F0E0EB0FF21DD2
:101AA000049178940395B091AF00B01708F4C6CFB5
:101AB00088DF87DFB091AE00B395B093AE00B091F0
:101AC000AE00BA3008F4B7CFFCDAF89420DFB8E003
:061AD000B1BD77DFBBCBC6
:00000001FF
